:100000000C949B050C94FC050C94FC050C94EE06DA
:100010000C94FC050C94FC050C94FC050C94FC055C
:100020000C94FC050C94FC050C9435100C940711F1
:100030000C941F1E0C94FC050C94FC050C94FC0500
:100040000C94FC050C94FC050C94FC050C94FC052C
:100050000C94FC050C94931E0C94FC050C94FC056C
:100060000C94FC050C94FC050C94FC050C94FC050C
:100070000C94FC050C94FC050C94FC050C94FC05FC
:100080000C94FC050C94FC050C94FC050C94FC05EC
:100090000C94FC050C94FC050C94FC050C94FC05DC
:1000A0000C94FC050C94FC050C94FC05830EAA0E24
:1000B000A20FAA0EA20FF60E190FA20F700F7F0F3C
:1000C0004F144F1479147914D414081516171617F1
:1000D0001F1516170A160A16D0161617E516031757
:1000E00080680169023A3B433C443D453E7E3F7394
:1000F0004041427A52484647506A6B514F291E1F71
:1001000020212223242526272D2E352A4903545524
:100110007C6C636D4A2B141A0815171C180C1213EB
:100120002F304C655F6061566E6F4D807804160706
:10013000090A0B0D0E0F33343128585C5D5E627076
:100140004B7153791D1B06190511103637387D7513
:10015000595A5B77760072397B2C7F4E64578080CA
:10016000253032580A007265736574206661696CC7
:100170003A2000253032580A006C61796F75743A64
:100180002000253032580A0072657365743A2000E9
:100190002000253032580020446F6E650A002E0082
:1001A0005265736574696E6720004C45443A20259A
:1001B0003032580A00556E6B6E6F776E206578741A
:1001C000726120636F6D6D616E643A202530325824
:1001D0000A006C61796F75740A004C454420616CAB
:1001E0006C206F66660A004C454420616C6C206F81
:1001F0006E0A00436C69636B204F66660A00436CAD
:1002000069636B204F6E0A0042656C6C204F666616
:100210000A0042656C6C204F6E0A0052657365746B
:100220000A0044656C6574653A2020202020205225
:10023000657365740A00496E736572743A202020F4
:100240002020204C61796F75740A005067446F77E5
:100250006E3A2020202020204C454420616C6C20E8
:100260004F66660A00506755703A202020202020F3
:1002700020204C454420616C6C204F6E0A00456E76
:10028000643A202020202020202020546F67676CB3
:100290006520436C69636B0A00486F6D653A2020E6
:1002A000202020202020546F67676C652042656CF9
:1002B0006C0A000A0A2D2D2D2D2D2053756E2063FA
:1002C0006F6E7665727465722048656C70202D2D96
:1002D0002D2D2D0A000A4B6579626F6172642073BF
:1002E000746172742E0A000A55534220636F6E6661
:1002F0006967757265642E0A000A0A544D4B3A65A7
:10030000363361666638372F4C5546410A0A002E4F
:1003100003530075006E0020006B006500790062D9
:10032000006F00610072006400200063006F006EC7
:100330000076006500720074006500720000000E17
:100340000374002E006D002E006B002E00000004D0
:1003500003090409027400040100A032090400002A
:1003600001030101000921110100012240000705DC
:10037000810308000A0904010001030102000921A8
:1003800011010001224D000705820308000A09043B
:1003900002000103000000092111010001223600C2
:1003A0000705830308000A09040300020300000094
:1003B0000921110100012222000705840320000108
:1003C000070504032000011201100100000008EDE0
:1003D000FE33330001010200010631FF0974A1015F
:1003E0000975150026FF009520750881020976150C
:1003F0000026FF00952075089102C005010980A123
:100400000185021601002637001A81002AB70075FF
:100410001095018100C0050C0901A1018503160199
:1004200000269C021A01002A9C0275109501810089
:10043000C005010902A1010901A10005091901294D
:10044000051500250195057501810295017503814A
:10045000010501093009311581257F950275088153
:100460000609381581257F950175088106050C0A56
:1004700038021581257F950175088106C0C00501E8
:100480000906A101050719E029E7150025019508CE
:100490007501810295017508810105081901290579
:1004A00095057501910295017503910105071900E4
:1004B00029FF150026FF00950675088100C0636FAF
:1004C0006E73756D65723A20253034580A00737961
:1004D0007374656D3A20253034580A000A002530BF
:1004E000325820006B6579626F6172643A20004C6B
:1004F00045443A20253032580A00253032583A20F7
:100500002530386225730A00722F63203031323370
:10051000343536370A00290A002575002F00257565
:10052000005D28002564002000256400200025646B
:100530000020002564007C0025303258006D6F7566
:1005400073656B6579205B62746E7C7820792076A8
:1005500020685D287265702F61636C293A205B000A
:100560006D6B5F776865656C5F74696D655F746FEF
:100570005F6D6178203D2025640A006D6B5F7768B0
:1005800065656C5F6D61785F7370656564203D20A3
:1005900025640A006D6B5F74696D655F746F5F6DD4
:1005A0006178203D2025640A006D6B5F6D61785F86
:1005B0007370656564203D2025640A006D6B5F697A
:1005C0006E74657276616C203D2025640A006D6B47
:1005D0005F64656C6179203D2025640A006D6B5F66
:1005E000776865656C5F74696D655F746F5F6D6179
:1005F00078203D2025640A006D6B5F776865656C27
:100600005F6D61785F7370656564203D2025640AC5
:10061000006D6B5F74696D655F746F5F6D617820ED
:100620003D2025640A006D6B5F6D61785F737065B6
:100630006564203D2025640A006D6B5F696E7465FA
:100640007276616C203D2025640A006D6B5F6465E5
:100650006C6179203D2025640A000A00257500366A
:100660003A20776865656C5F74696D655F746F5F6C
:100670006D61783A20000A00257500353A207768C8
:1006800065656C5F6D61785F73706565643A2000C5
:100690000A00257500343A2074696D655F746F5FD8
:1006A0006D61783A20000A00257500333A206D61AB
:1006B000785F73706565643A20000A002575003222
:1006C0003A20696E74657276616C286D73293A20E0
:1006D000000A00257500313A2064656C6179282A8A
:1006E00031306D73293A20000A092D2056616C754E
:1006F0006573202D0A004D3E004D25643E20003FCD
:10070000007365742064656661756C740A00433E0D
:10071000200077686572652064656C74613A2063B7
:100720007572736F723D25642C20776865656C3D2A
:1007300025640A53656520687474703A2F2F656EBE
:100740002E77696B6970656469612E6F72672F77A8
:10075000696B692F4D6F7573655F6B6579730A00FF
:100760000A092D204D6F7573656B6579202D0A453B
:1007700053432F713A09717569740A313A096465F6
:100780006C6179282A31306D73290A323A09696E11
:1007900074657276616C286D73290A333A096D614C
:1007A000785F73706565640A343A0974696D655FD2
:1007B000746F5F6D61780A353A09776865656C5FBB
:1007C0006D61785F73706565640A363A09776865AC
:1007D000656C5F74696D655F746F5F6D61780A0A3F
:1007E000703A097072696E742076616C7565730A6F
:1007F000643A097365742064656661756C74730A84
:1008000075703A092B310A646F776E3A092D310AF7
:10081000706775703A092B31300A7067646F776EB4
:100820003A092D31300A0A7370656564203D2064F1
:10083000656C7461202A206D61785F7370656564F2
:10084000202A2028726570656174202F2074696DDC
:10085000655F746F5F6D6178290A003F004D3E202F
:1008600000433E20004C25640A000A092D20436FF6
:100870006E736F6C65202D0A4553432F713A0971D1
:100880007569740A6D3A096D6F7573656B65790AE0
:10089000000A092D204D61676963202D0A643A0919
:1008A00064656275670A783A096465627567206DE8
:1008B00061747269780A6B3A096465627567206BC6
:1008C0006579626F6172640A6D3A09646562756781
:1008D000206D6F7573650A763A0976657273696F74
:1008E0006E0A733A097374617475730A633A096323
:1008F0006F6E736F6C65206D6F64650A302D343ACE
:10090000096C61796572302D34284631302D4634BA
:10091000290A506175733A09626F6F746C6F616474
:1009200065720A003F0074696D65725F726561648B
:10093000333228293A202530346C580A006B657907
:10094000626F6172645F69646C653A2025580A00C1
:100950006B6579626F6172645F70726F746F636FE1
:100960006C3A2025580A00686F73745F6B65796272
:100970006F6172645F6C65647328293A2025580A98
:10098000000A092D20537461747573202D0A0047E5
:1009900043433A20352E342E30204156522D4C49B7
:1009A00042433A20322E302E30204156525F41527F
:1009B00043483A20617672350A004F5054494F4EF1
:1009C000533A204C554641204D4F5553454B4559C0
:1009D0002045585452414B455920434F4E534F4C9C
:1009E0004520434F4D4D414E44204B45594D4150BC
:1009F0005F53454354494F4E20424F4F544C4F4153
:100A00004445525F53495A450A004255494C443ABD
:100A1000206536336166663837202831333A3537FA
:100A20003A3233204170722020392032303230295E
:100A30000A005649443A2030784645454428742EE9
:100A40006D2E6B2E29205049443A203078333333B1
:100A5000332853756E206B6579626F617264206311
:100A60006F6E76657274657229205645523A203051
:100A700078303130300A00444553433A20636F6E7A
:100A800076657274732053756E206B6579626F6141
:100A900072642070726F746F636F6C20696E746F14
:100AA000205553420A000A092D2056657273696F5A
:100AB0006E202D0A000A6D6F7573653A206F6666A9
:100AC0000A000A6D6F7573653A206F6E0A000A6B33
:100AD0006579626F6172643A206F66660A000A6B1C
:100AE0006579626F6172643A206F6E0A000A6D6107
:100AF000747269783A206F66660A000A6D617472D2
:100B000069783A206F6E0A000A64656275673A2058
:100B10006F6E0A000A64656275673A206F66660A3E
:100B2000000A0A626F6F746C6F616465722E2E2EFC
:100B30002000433E200011241FBECFEFDAE0DEBFCD
:100B4000CDBF04B603FE41C080916A0390916B0350
:100B5000A0916C03B0916D038730904BA740B04BD0
:100B6000A1F510926A0310926B0310926C0310921D
:100B70006D0314BE0FB6F894A8958091600088614B
:100B800080936000109260000FBE109201081092D6
:100B90000008E3E0F0E089E080935700E491E695F7
:100BA000E370E150E33040F4F0E0EE0FFF1FE25D50
:100BB000FE4F8081918102C080E090E1E0E0F0E8AA
:100BC000E81BF90BF695E795099511E0A0E0B1E077
:100BD000EAEEFDE402C005900D92AE33B107D9F7FD
:100BE00023E0AEE3B1E001C01D92AA36B207E1F7FF
:100BF0000E94A10B0C94F3260C940000FF93EF933A
:100C0000E0913E01F0913F01309709F00995EF9195
:100C1000FF910895FC018591803011F0EFDFFBCF4B
:100C20000895FF27E0E230E247FF0CC0419597FFAF
:100C300009C0EDE26095709580959095611D711DDC
:100C4000811D911D27FF02C0219530E350E2AA27A4
:100C5000660F771F881F991FAA1FA41710F0A41BE7
:100C600063955A95A9F7AA3008F0A95FA05DAF93E4
:100C7000F395611571058105910541F7ED3211F488
:100C8000EF93F395F21718F43F93F395FBCF8F9101
:100C9000B5DFFA95E1F70895E991F99185918030F2
:100CA00021F0853219F0AADFF9CF089520E0E89409
:100CB00055915532C1F3503311F4689455915A331C
:100CC00048F4505390F3220F022E220F220F200DD2
:100CD000250FF4CF0EF4219589919991533619F38C
:100CE000533729F1533559F1BC0188279927E894E6
:100CF0005C3621F48991999168945591543639F470
:100D000046EF7EF077FF0DC08FEF9FEF0AC055379B
:100D10004AE039F0583540E121F0523642E009F01E
:100D20000895FF93EF937DDFEF91FF91B7CFFF938E
:100D3000EF93FC0181918030B9F360DFFBCFFF932B
:100D4000EF9368DFF1CFDF93CF93CDB7DEB7259672
:100D5000A3DFCF91DF91089552985A9AE9E6F0E027
:100D6000808180638083EA9A7894539A5B9808958F
:100D70002091400180914101821761F030E0F9013A
:100D8000EE5BFE4F80812F5F3F4F2770332720930C
:100D90004001089580E008955B9AE3E0FDE031971B
:100DA000F1F700C0000028E030E091E0482F49232F
:100DB00011F05B9801C05B9AE3E0FDE03197F1F739
:100DC00000C00000990F2150310981F75B9883E042
:100DD0009DE00197F1F700C0000008951F920F9267
:100DE0000FB60F9211242F933F934F935F938F93DE
:100DF0009F93EF93FF938FE796E00197F1F700C081
:100E0000000088E090E021E040E0E3E0FDE0319781
:100E1000F1F700C000004A9B422B220F0197A9F76F
:100E200083E09DE00197F1F700C00000809141014F
:100E300090E09C012F5F3F4F277033275091400176
:100E4000521731F0FC01EE5BFE4F408320934101CD
:100E500084E08CBBFF91EF919F918F915F914F91B7
:100E60003F912F910F900FBE0F901F901895569A9B
:100E70005E9A0E94AC06EAE4F1E0119221E0EA35C4
:100E8000F207D9F780EA91E00E940A068EE991E024
:100E90000E940A060E94B8068111FCCF81E00E94E0
:100EA000CC068FEF99E628E1815090402040E1F791
:100EB00000C000000E94B8068F3F41F78FEF99E60F
:100EC00028E1815090402040E1F700C000000E94DE
:100ED000B8068430D9F687E991E00E940A065E9848
:100EE00008951F93CF93DF930E94B806C82F8823DD
:100EF00009F476C080914C0380FF0CC01F92CF9301
:100F000082E991E09F938F930E94A3060F900F9028
:100F10000F900F9080914C0380FF04C080E991E016
:100F20000E940A06CF3709F45DC0B8F4CE3709F045
:100F300061C086E691E00E940A062FEF89E698E1FB
:100F4000215080409040E1F700C000000E94B806A8
:100F50001F928F9380E691E03BC0CE3F31F1CF3FAF
:100F600009F048C088E891E00E940A062FEF89E660
:100F700098E1215080409040E1F700C000000E94BD
:100F8000B806C82F1F928F9382E891E09F938F93AA
:100F90000E94A3060F900F900F900F90C43001F5A0
:100FA0000E9451110E9435081BC089E791E00E9400
:100FB0000A062FEF89E698E1215080409040E1F742
:100FC00000C000000E94B8061F928F9383E791E053
:100FD0009F938F930E94A3060F900F900F900F90F6
:100FE00080E039C0EAE4F1E0119221E0EA35F2074D
:100FF000D9F7F6CF1C2F1770DC2FD695D695D6953E
:10100000C7FF15C0DF70612F8D2F0E94B812882393
:1010100009F1ED2FF0E0E65BFE4F81E090E001C0CA
:10102000880F1A95EAF780959081892312C0612F65
:101030008D2F0E94B81281110DC0ED2FF0E0E65BFC
:10104000FE4F81E090E001C0880F1A95EAF7908189
:10105000892B80838C2FDF91CF911F910895E82FEA
:10106000F0E0E65BFE4F80810895CF93C82FC170FA
:1010700083FDC26082FDC46081FDC8601F928F93B2
:101080008AEA91E09F938F930E94A3068EE00E94CC
:10109000CC060F900F900F900F908C2FCF910C9447
:1010A000CC06CF938A3409F440C048F48833D1F099
:1010B000893409F46DC08B3009F073C013C08C34CF
:1010C00071F108F45CC08D3409F443C08E3409F02A
:1010D00068C08AED91E00E940A068EE00E94CC066C
:1010E00080E05BC083EB92E00E940A0689E992E00F
:1010F0000E940A068EE792E00E940A0685E692E0C8
:101100000E940A068BE492E00E940A0686E392E0BF
:101110000E940A0682E292E00E940A064EC08BE11B
:1011200092E00E940A0681E038C0C0915B0181E034
:10113000C827C0935B01CC2331F082E192E00E948A
:101140000A0682E013C088E092E00E940A0683E06B
:1011500024C0C0915A0181E0C827C0935A01CC2312
:1011600041F08EEF91E00E940A068AE00E94CC06D0
:1011700025C083EF91E00E940A068BE00EC087EE47
:1011800091E00E940A068EE00E94CC068FEF05C017
:1011900082ED91E00E940A068FE00E94CC06C1E039
:1011A0000DC01F928F9385EB91E09F938F930E94C8
:1011B000A3060F900F900F900F90C0E08C2FCF914F
:1011C0000895809168020895CF93DF9300D01F9215
:1011D000CDB7DEB79C0180916103843019F593E0AF
:1011E00099833B832A839093E9008FEF9091E800E5
:1011F000815095FD06C095ED9A95F1F7000081119B
:10120000F5CF8091E80085FF0DC040E050E063E03D
:1012100070E0CE0101960E94500D8091E8008E771B
:101220008093E8000F900F900F90DF91CF91089579
:10123000CF93DF9300D01F92CDB7DEB7209161032B
:10124000243031F522E02983805891099B838A83D9
:1012500083E08093E9008FEF9091E800815095FD45
:1012600006C095ED9A95F1F700008111F5CF8091B8
:10127000E80085FF0DC040E050E063E070E0CE0183
:1012800001960E94500D8091E8008E778093E800CF
:101290000F900F900F90DF91CF91089520916103EF
:1012A0002430F1F422E02093E9002FEF3091E800A0
:1012B000215035FD06C035ED3A95F1F700002111BA
:1012C000F5CF2091E80025FF0BC040E050E065E03D
:1012D00070E00E94500D8091E8008E778093E800C6
:1012E0000895CF93DF9320916103243049F521E0E5
:1012F0002093E90021E8215059F03091E80035FDB4
:1013000007C0EFE3F1E03197F1F700C00000F3CF41
:101310002091E80025FF14C0EC0140E050E068E0B7
:1013200070E00E94500D8091E8008E778093E80075
:1013300088E0FE01A0E6B2E001900D928A95E1F707
:10134000DF91CF910895CF93C0915E01C1110BC081
:101350000E945D1E643C79408105910520F081E08A
:1013600080935E01C1E08C2FCF910895FF920F937F
:101370001F93CF93DF93D82F0FB607FE83C08091C2
:101380006103843081F08091030190E00196209107
:10139000050130E0822393232091040130E082177D
:1013A000930709F0CDC00E94A309811110C080915C
:1013B000030190E001962091050130E08223932300
:1013C0002091040130E08217930709F0B9C00E9410
:1013D000511E8C01C091E900CF709091EC00892FD3
:1013E000817090FD80E8C82B84E08093E90085E05F
:1013F000F82E8091EB0085FD42C08091EB0080FFCC
:101400003EC08091EE0087FF3AC080910401909128
:101410000301981709F457C09091E80095FF8EC01A
:10142000E0910101F0910201E80FF11D20818F5F31
:10143000909105018923809304012093F10080910C
:10144000E80085FDE2CF8091E80080FFDECF80914B
:10145000E8008E778093E800F0920001D6CF80916B
:10146000030190E001962091050130E0822393234F
:101470002091040130E08217930709F44CC0CF702B
:10148000C093E90040910301842F90E001962091E0
:10149000050130E0822393232091040130E082177C
:1014A000930709F450C0E0910101F0910201E40FAB
:1014B000F11DD083809103018F5F909105018923F5
:1014C0008093030140C08091E80085FF37C0D0932E
:1014D000F10021E03091F3008091F20090E0932B35
:1014E000892B91F08091E80080FF0EC08091E80088
:1014F00085FF03C01092F100F9CF8091E8008E774C
:101500008093E800F0920001222309F4A8CFCF7065
:10151000C093E90018C080910001882309F4AFCF7F
:101520000E94511E9C018017910711F4890161CF1F
:1015300090910001915090930001F8CF20E0CACF24
:1015400040910301B0CF80E0DF91CF911F910F91C7
:10155000FF90089580916003811104C00E94BA0F2A
:101560000C9417100895109260030895089542E0B6
:1015700061EC81E00E94C90C42E061EC82E00E94D3
:10158000C90C42E061EC83E00E94C90C42E261ECCC
:1015900084E00C94C90C80916303833009F453C038
:1015A00030F4813071F0823009F48CC008958A30B3
:1015B00009F478C08B3009F45EC0893009F09AC014
:1015C00020C080916203813A09F094C08091E800C4
:1015D000877F8093E8008091660390916703892B51
:1015E00021F468E080E692E003C060E080E090E0F3
:1015F00070E00E949B0D8091E8008B778093E8005B
:10160000089580916203813209F074C0809166036D
:1016100090916703892B09F06DC08091E800877F66
:101620008093E8008091E80082FD05C0809161030D
:101630008111F8CF5FC08091F100809368028091A2
:10164000E8008B7753C080916203813A09F052C061
:101650008091660390916703892B09F04BC08091BC
:10166000E800877F8093E8008091E80080FFFCCF4E
:101670008091100136C0809162038132D9F580914A
:10168000660390916703892BA9F58091E800877F15
:101690008093E8000E94FE0C809164038093100107
:1016A0000C94FF1380916203813221F58091E80050
:1016B000877F8093E8000E94FE0C809165038093F1
:1016C0006902089580916203813AA1F48091E80053
:1016D000877F8093E8008091E80080FFFCCF8091B5
:1016E00069028093F1008091E8008E778093E80092
:1016F0000C94FE0C08958091680280935F01109213
:1017000068020E94B6120C94FF130C947B0B0E948B
:10171000DE1D80915F03882329F00E94071E81113E
:101720000C94B30C08950E941B1E80915F0180935E
:10173000680208950C94930B08950C949C0B0C94E0
:101740009C0BCF9384B7877F84BF0FB6F894A8957E
:1017500080916000886180936000109260000FBEED
:1017600090E080E80FB6F894809361009093610058
:101770000FBE86EB99E00E94B11D86E091E00E94C9
:101780004C1189EF92E00E940A060E949F0B0E9472
:101790000B120E94BA0F0E94171078940E940D122B
:1017A00080916103843019F00E949C0BF9CF87EE81
:1017B00092E00E940A060E949D0B85ED92E00E9435
:1017C0000A06C4E080916103853019F40E94870BFA
:1017D000F9CF0E9411122091E4003091E500809130
:1017E0005C0190915D012817390761F38091E40055
:1017F0009091E50090935D0180935C010E94A309A4
:10180000882301F3809161038430E1F68091E9003F
:101810008F702091EC00922F917020FD90E8892B21
:10182000C093E9009091EB0090FF43C09091EE00CF
:1018300097FF3FC09091040120910301291709F1FE
:101840002091E80025FF1DC0E0910101F091020107
:10185000E90FF11D30819F5F209105019223909344
:1018600004013093F1009091E80095FDE3CF909151
:10187000E80090FFDFCF9091E8009E779093E8001A
:10188000D9CF9091F3002091F20030E0392B232B37
:1018900081F09091E80090FF0CC09091E80095FFD6
:1018A00003C01092F100F9CF9091E8009E779093D9
:1018B000E8008F708093E90085CF292F33272330EC
:1018C0003105C9F060F42130310581F02230310555
:1018D00009F041C084E790E023E533E040C02132C5
:1018E0003105E1F02232310531F135C082E190E07D
:1018F00027EC33E034C099278130910549F028F076
:10190000029749F5EFE0F3E005C0EFE4F3E002C031
:10191000EFE3F3E0849190E09F0121C06430710512
:10192000D0F4660F771FFB01EB5DFE4F2081318104
:1019300089E090E014C06430710568F4FB01EE0F9B
:10194000FF1FE35EFE4F20813181FB01E75EFE4F0A
:10195000808190E004C080E090E020E030E0FA0177
:1019600031832083089580E189BD82E189BD09B476
:1019700000FEFDCF8091D8008F7D8093D8008091AC
:10198000E00082608093E0008091E00081FDFCCF68
:101990000895982F973068F59093E900981739F0DB
:1019A0007091EC002091ED005091F00003C0242FC5
:1019B000762F50E021FD02C09F5FECCF3091EB000D
:1019C0003E7F3093EB003091ED003D7F3093ED0092
:1019D0003091EB0031603093EB007093EC0020937A
:1019E000ED005093F0002091EE0027FDE5CF80E060
:1019F00008958F708093E90081E0089580916203DB
:101A000087FF11C08091E80082FD05C080916103CD
:101A10008111F8CF11C08091E8008B770BC08091C5
:101A20006103882349F08091E80080FFF8CF80911E
:101A3000E8008E778093E80008952091E4003091CB
:101A4000E50095E64091EC00842F817040FF23C0B3
:101A50008091E80080FD1DC080916103882399F08A
:101A6000853099F08091EB0085FD11C04091E40034
:101A70005091E5002417350729F3915011F09A0190
:101A8000E1CF84E0089582E0089583E0089581E045
:101A9000089580E008954091E80042FFDDCF089569
:101AA000CF92DF92EF92FF920F931F93CF93DF932A
:101AB000EC018B017A010E941D0D811133C0E114EC
:101AC000F10439F0F70180819181081B190BC80FCF
:101AD000D91FC12CD12C0115110519F18091E800F5
:101AE00085FD16C08091E8008E778093E800E114B0
:101AF000F10449F0F70180819181C80ED91ED1828D
:101B0000C08285E00FC00E941D0D882321F30AC00A
:101B100089918093F10001501109FFEFCF1ADF0A7C
:101B2000DACF80E0DF91CF911F910F91FF90EF907E
:101B3000DF90CF90089520916803309169032617B4
:101B4000370748F06115710539F42091E8002E77C8
:101B50002093E80001C0B901FC0120E06115710586
:101B600079F1809161038823F1F18530F1F1809161
:101B7000E80083FD3CC08091E80082FD2EC080918A
:101B8000E80080FFEBCF2091F3008091F20090E01D
:101B9000922B6115710551F08830910538F421912F
:101BA0002093F100615071090196F3CF21E008976D
:101BB00009F020E08091E8008E778093E800CECF96
:101BC0002111CFCF0AC080916103882361F0853055
:101BD00061F08091E80083FD0AC08091E80082FFF7
:101BE000F2CF80E0089582E0089583E0089581E0D7
:101BF000089520916803309169032617370748F04C
:101C00006115710539F42091E8002E772093E800E2
:101C100001C0B901FC0120E06115710591F18091CD
:101C20006103882309F440C0853009F43FC08091E6
:101C3000E80083FD3DC08091E80082FD2FC08091C7
:101C4000E80080FFE9CF2091F3008091F20090E05E
:101C5000922B6115710559F08830910540F424915B
:101C60002093F1003196615071090196F2CF21E085
:101C7000089709F020E08091E8008E778093E800D3
:101C8000CBCF2111CCCF0AC080916103882361F0B2
:101C9000853061F08091E80083FD0AC08091E80002
:101CA00082FFF2CF80E0089582E0089583E00895F6
:101CB00081E008951F93CF93DF93CDB7DEB7AA9746
:101CC0000FB6F894DEBF0FBECDBFE2E6F3E0809121
:101CD000F100819323E0EA36F207C9F70E94CB0AAC
:101CE0008091E80083FF2EC180916203909163038D
:101CF000492F50E04A30510508F024C1FA01EA5A50
:101D0000FF4F0C94D926803821F0823809F01AC18F
:101D100008C080915E0390915F03992389F08260EF
:101D20000FC0809166038F70873008F00BC18093DD
:101D3000E9008091EB0085FB882780F91092E9008B
:101D40009091E800977F9093E8008093F1001092C3
:101D5000F100D1C0282F2D7F09F0F4C0882319F09D
:101D6000823061F0EFC080916403813009F0EAC0F5
:101D7000933009F080E080935F032EC0809164036C
:101D800081112AC0809166038F702FEF280F2630B3
:101D900008F0D8C08093E9002091EB0020FF1CC020
:101DA000933021F48091EB00806214C09091EB009D
:101DB00090619093EB0021E030E0A90102C0440F54
:101DC000551F8A95E2F74093EA001092EA0080914D
:101DD000EB0088608093EB001092E9008091E800AE
:101DE000877F8093E8000E94FE0CACC08111AAC0DE
:101DF000109164031F778091E3008078812B80939A
:101E0000E3008091E800877F8093E8000E94FE0C49
:101E10008091E80080FFFCCF8091E3008068809390
:101E2000E300111102C082E001C083E080936103EE
:101E300089C08058823008F085C0809164039091F9
:101E400065038C3D53E0950779F583E08A838AE248
:101E500089834FB7F894DE01139620E03EE051E20B
:101E6000E32FF0E050935700E49120FF03C0E29588
:101E7000EF703F5FEF708E2F90E0EA3010F0C79662
:101E800001C0C0968D939D932F5F243149F74FBFBA
:101E90008091E800877F8093E8006AE270E0CE01DD
:101EA00001960E949B0D16C06091660370916703B6
:101EB000AE014F5F5F4F0E945D0CBC01892B09F49E
:101EC00041C09091E800977F9093E80089819A81C2
:101ED0000E94F90D8091E8008B778093E80032C072
:101EE000803881F58091E800877F8093E8008091B9
:101EF0005D038093F1008091E8008E7772CF8111AD
:101F000021C0809164039091650399270297D4F4CE
:101F10008091E800877F8093E8008091640380933C
:101F20005D030E94FE0C80915D03811106C08091CB
:101F3000E30087FD02C081E001C084E0809361037B
:101F40000E94B70A8091E80083FF0AC08091E800F0
:101F5000877F8093E8008091EB0080628093EB00A4
:101F6000AA960FB6F894DEBF0FBECDBFDF91CF911A
:101F70001F9108950E9428100E943010E0EEF0E0BA
:101F8000808181608083E8EDF0E080818F778083BD
:101F900019BCA7EDB0E08C918E7F8C9380818F7EF1
:101FA00080831092600308950F931F93CF93DF9364
:101FB0000E9428100E943010C8EDD0E088818F77F1
:101FC000888388818068888388818F7D888319BC15
:101FD0001092610310925D0310925F0310925E03F2
:101FE00000EE10E0F80180818B7F80838881816022
:101FF000888342E060E080E00E94C90CE1EEF0E0FE
:1020000080818E7F8083E2EEF0E08081816080833A
:10201000808188608083F80180818E7F80838881C1
:1020200080618883DF91CF911F910F910895E8ED32
:10203000F0E080818F7E8083E7EDF0E08081816039
:10204000808384E082BF81E0809360030C94D40F8E
:10205000E8EDF0E080818E7F80831092E2000895A9
:102060001092DA001092E10008951F920F920FB6BD
:102070000F9211242F933F934F935F936F937F930E
:102080008F939F93AF93BF93EF93FF938091E10062
:1020900082FF0BC08091E20082FF07C08091E100C7
:1020A0008B7F8093E1000E944B118091DA0080FFCA
:1020B0001FC08091D80080FF1BC08091DA008E7F06
:1020C0008093DA008091D90080FF0DC080E189BD46
:1020D00082E189BD09B400FEFDCF81E080936103F8
:1020E0000E94AA0A05C019BC109261030E94B30A9B
:1020F0008091E10080FF19C08091E20080FF15C04F
:102100008091E2008E7F8093E2008091E200806106
:102110008093E2008091D80080628093D80019BC3F
:1021200085E0809361030E94850B8091E10084FF2C
:1021300030C08091E20084FF2CC080E189BD82E143
:1021400089BD09B400FEFDCF8091D8008F7D8093BA
:10215000D8008091E1008F7E8093E1008091E200C1
:102160008F7E8093E2008091E20081608093E200A4
:1021700080915D03882311F084E007C08091E30023
:1021800087FD02C081E001C083E0809361030E946B
:102190009A0B8091E10083FF29C08091E20083FFC8
:1021A00025C08091E100877F8093E10082E08093E9
:1021B000610310925D038091E1008E7F8093E100C6
:1021C0008091E2008E7F8093E2008091E200806146
:1021D0008093E20042E060E080E00E94C90C8091C0
:1021E000F00088608093F0000E94B60AFF91EF91A2
:1021F000BF91AF919F918F917F916F915F914F911F
:102200003F912F910F900FBE0F901F9018951F9226
:102210000F920FB60F9211242F933F934F935F931A
:102220006F937F938F939F93AF93BF93CF93DF93DE
:10223000EF93FF93C091E900CF708091EC00D82F0D
:10224000D17080FDD0E81092E9008091F000877F86
:102250008093F00078940E945A0E1092E9008091C9
:10226000F00088608093F000CD2BCF70C093E90020
:10227000FF91EF91DF91CF91BF91AF919F918F919E
:102280007F916F915F914F913F912F910F900FBE72
:102290000F901F901895089590936F0280936E028F
:1022A0000895E0916E02F0916F02309721F0019055
:1022B000F081E02D099480E00895EF92FF920F9352
:1022C0001F93CF93DF93E0916E02F0916F023097EE
:1022D000B1F18C010280F381E02D099580914C03CE
:1022E00082FF2DC080FF04C084EE94E00E940A06A5
:1022F000E80118E08EEDE82E84E0F82E80914C0382
:1023000080FF0BC088811F928F93FF92EF920E94F3
:10231000A3060F900F900F900F901150219611115E
:10232000EDCF80914C0380FF0AC08CED94E0DF91EB
:10233000CF911F910F91FF90EF900C940A06DF91BF
:10234000CF911F910F91FF90EF900895E0916E0251
:10235000F0916F02309721F00480F581E02D09940F
:102360000895CF93DF9320916C0230916D0228176E
:10237000390709F190936D0280936C02E0916E022F
:10238000F0916F023097B9F0EC010680F781E02DF3
:10239000099580914C0382FF0EC080FF0CC0DF9333
:1023A000CF938EEC94E09F938F930E94A3060F909F
:1023B0000F900F900F90DF91CF910895CF93DF93FF
:1023C00020916A0230916B022817390709F1909326
:1023D0006B0280936A02E0916E02F0916F02309777
:1023E000B9F0EC010084F185E02D099580914C0352
:1023F00082FF0EC080FF0CC0DF93CF938EEB94E082
:102400009F938F930E94A3060F900F900F900F90B1
:10241000DF91CF9108950C94B7120E94481E0C943E
:102420003707BF92CF92DF92EF92FF920F931F93E5
:10243000CF93DF9300D000D01F92CDB7DEB70E94BC
:10244000710701E712E0F12C8F2D0E942F08B82EA2
:10245000F801C080C82639F4F3940F5F1F4FF0E1F4
:10246000FF12F2CF30C080914C0381FD0E94CC124C
:10247000D12CEE24E3948C2D8E21F9F0D982FA82AE
:1024800091E08B2D8E2109F490E09B830E94511ED8
:102490008160782F9D838C8349815A816B818D81E6
:1024A0000E94021349815A816B817C818D810E9437
:1024B000C91DF80180818E258083D394EE0CF8E04D
:1024C000DF12D9CFC9CF8FEF89838A831B820E9405
:1024D000511E8160782F9D838C8349815A816B8145
:1024E0008D810E9402130E94C81D0E940F210E942C
:1024F000511190917002891741F10E9451118093FE
:10250000700290914C0392FF0EC090FF0CC01F927E
:102510008F938FEE94E09F938F930E94A3060F906A
:102520000F900F900F90809170020F900F900F906E
:102530000F900F90DF91CF911F910F91FF90EF902F
:10254000DF90CF90BF900C94DA1D0F900F900F90FA
:102550000F900F90DF91CF911F910F91FF90EF900F
:10256000DF90CF90BF9008950C943508089508959A
:10257000CF93C62F0E942F0821E030E002C0220F27
:10258000331FCA95E2F790E02823392381E0232BFB
:1025900009F480E0CF910895EF92FF920F931F937B
:1025A000CF93DF9388E095E00E940A06C0E0D0E078
:1025B0008DE2E82E81E0F82E0AEF14E08C2F0E94C5
:1025C0002F080E94B61DFF92EF921F928F93DF9308
:1025D000CF931F930F930E94A30621968DB79EB7AA
:1025E00008960FB6F8949EBF0FBE8DBFC031D105BF
:1025F00029F7DF91CF911F910F91FF90EF900895F0
:1026000008950895CF93DF93CDB7DEB72B970FB61C
:10261000F894DEBF0FBECDBF942F4F83252F588770
:1026200069877A878B874A855B85452B31F02F3FF9
:1026300031F481E09F3F19F403C081E001C080E0E4
:1026400080FD07C04F81588569857A858B850E94FA
:10265000C91DDE01119686E0FD0111928A95E9F708
:1026600085E0FE01379601900D928A95E1F7498148
:102670005A816B817C818D819E810E942B1A2B96C1
:102680000FB6F894DEBF0FBECDBFDF91CF91089596
:10269000CF93882309F465C0C82F8CEF8C0F813A43
:1026A00020F080E58C0F8E3248F48C2F0E94372466
:1026B000811157C08C2F0E94131D0CC080E28C0F1B
:1026C000883058F4C77081E001C0880FCA95EAF7D6
:1026D0000E94511DCF910C948B1D8BE58C0F833084
:1026E00078F4C53A29F0C63A31F083E890E005C0A5
:1026F00081E890E002C082E890E0CF910C94B111A3
:1027000088E58C0F853168F5C83A89F0C93A91F0AF
:10271000CA3A99F0CB3AA1F0CC3AA9F0CD3AB1F04F
:10272000CE3AB9F0CF3AC1F080E090E017C082EE27
:1027300090E014C089EE90E011C08AEE90E00EC0E7
:1027400085EB90E00BC086EB90E008C083EB90E057
:1027500005C084EB90E002C087EB90E0CF910C9431
:10276000DE11CF910895882349F19CEF980F913A9B
:1027700020F090E5980F9E3218F40E94301D0DC095
:1027800090E2980F983058F4877091E001C0990F4B
:102790008A95EAF7892F0E94571D0C948B1D9BE5A3
:1027A000980F933020F480E090E00C94B111885A97
:1027B000853120F480E090E00C94DE1108958823A8
:1027C00021F00E94511D0C948B1D0895882321F047
:1027D0000E94571D0C948B1D08950E94711D0E942C
:1027E000401D0E948B1D0E94B4210E94822080E027
:1027F00090E00E94B11180E090E00C94DE110E9404
:10280000611D0C94ED13CF92DF92EF92FF920F9324
:102810001F93CF93DF9300D000D01F92CDB7DEB7C8
:102820006C010E94DC1D811101C385E0F601DE010F
:10283000119601900D928A95E1F7F6014081518140
:10284000238134812115310531F05F3F31F481E07E
:102850004F3F19F403C081E001C080E080FDE6C273
:10286000F601F280E580E2948FE0E82249835A8302
:10287000FB82722F3D832C836F2D8D810E948F1CD4
:102880008C010E948E1C0E947E1BE12FE295EF704E
:102890008E2F90E0FC01E05AFF4F0C94D926812F37
:1028A000807F1F70882311F01295107FFF2049F060
:1028B000112309F452C2812F0E94641D0E948B1DB6
:1028C0004CC2802F0E94B313112309F4AFC2812F91
:1028D0000E946A1D0F900F900F900F900F90DF9144
:1028E000CF911F910F91FF90EF90DF90CF900C94BC
:1028F0008B1D812F807F1F70803211F01295107F09
:10290000002319F0013009F12BC0FF20A9F0EE20BF
:1029100059F1F1E0812FEF1228C00F900F900F9026
:102920000F900F90DF91CF911F910F91FF90EF903B
:10293000DF90CF900C94741DEE2021F021E0E21680
:1029400009F474C20E94771D2DC0FF20E9F085E0D4
:102950008E1508F46BC20E944E1D812329F022C0FF
:10296000FF20F1F0E11015C0812F0F900F900F9014
:102970000F900F90DF91CF911F910F91FF90EF90EB
:10298000DF90CF900C94DF1394E09E1508F44EC2B4
:1029900009C0F601858180FFE0C18F708583E4CF97
:1029A000E110EEC1812F61C1812F869586958370DC
:1029B00019F08130B9F03AC2FF2019F0C8019370C4
:1029C00002C080E090E00F900F900F900F900F905A
:1029D000DF91CF911F910F91FF90EF90DF90CF90FB
:1029E0000C94B111FF2019F0C801937002C080E06F
:1029F00090E00F900F900F900F900F90DF91CF917C
:102A00001F910F91FF90EF90DF90CF900C94DE110B
:102A1000802FFF2019F00E94951F02C00E94FD1F09
:102A20000F900F900F900F900F90DF91CF911F910B
:102A30000F91FF90EF90DF90CF900C948220812F28
:102A4000837009F070C0F110F1C1202F22952695F6
:102A50002770220F220F602F6F70862F90E0A0E06A
:102A6000B0E06C017D01022E04C0CC0CDD1CEE1C1C
:102A7000FF1C0A94D2F704FF12C08FE090E0A0E0A0
:102A8000B0E004C0880F991FAA1FBB1F2A95D2F778
:102A9000BC01CD01609570958095909503C060E074
:102AA00070E0CB011695169513701230B1F040F519
:102AB0006C297D298E299F29113031F10F900F90BB
:102AC0000F900F900F90DF91CF911F910F91FF907A
:102AD000EF90DF90CF900C94A31B6C297D298E2959
:102AE0009F290F900F900F900F900F90DF91CF9133
:102AF0001F910F91FF90EF90DF90CF900C94BD1B32
:102B00000E94A31BC701B6010F900F900F900F906A
:102B10000F90DF91CF911F910F91FF90EF90DF9079
:102B2000CF900C94891BFF2019F0812F817001C078
:102B30008695882309F47AC1202F2295269527703F
:102B4000220F220F602F6F70862F90E0A0E0B0E080
:102B50006C017D01022E04C0CC0CDD1CEE1CFF1CA0
:102B60000A94D2F704FF12C08FE090E0A0E0B0E03A
:102B700004C0880F991FAA1FBB1F2A95D2F7BC015A
:102B8000CD01609570958095909503C060E070E0F0
:102B9000CB011695169513701230B1F040F56C29E3
:102BA0007D298E299F29113031F10F900F900F90C0
:102BB0000F900F90DF91CF911F910F91FF90EF90A9
:102BC000DF90CF900C946A1C6C297D298E299F2957
:102BD0000F900F900F900F900F90DF91CF911F915A
:102BE0000F91FF90EF90DF90CF900C947C1C0E948F
:102BF0006A1CC701B6010F900F900F900F900F90B5
:102C0000DF91CF911F910F91FF90EF90DF90CF90C8
:102C10000C94581C003FC1F128F480E4800F8032EE
:102C200050F096C0023F09F45EC008F449C0033F6B
:102C300009F46CC08DC0F02FF071EF2E812F8F71D1
:102C4000FF2051F00E94F11B802FEE2019F0829599
:102C5000807F8BCE8F7089CE0E94121C802FEE2039
:102C600019F08295807F01C08F700F900F900F90A8
:102C70000F900F90DF91CF911F910F91FF90EF90E8
:102C8000DF90CF900C94E613FF20A9F024E02E15DE
:102C900008F4CCC0812F8F710F900F900F900F9080
:102CA0000F90DF91CF911F910F91FF90EF90DF90E8
:102CB000CF900C94371C85E08E1508F4B7C0EACF8E
:102CC000FF2099F0812F8F710F900F900F900F9030
:102CD0000F90DF91CF911F910F91FF90EF90DF90B8
:102CE000CF900C94F11BFF2069F3812F8F710F900F
:102CF0000F900F900F900F90DF91CF911F910F9138
:102D0000FF90EF90DF90CF900C94121CFF2089F081
:102D1000812F8F710F900F900F900F900F90DF9178
:102D2000CF911F910F91FF90EF90DF90CF900C9477
:102D3000DC1B0F900F900F900F900F90DF91CF91B1
:102D40001F910F91FF90EF90DF90CF900C94D71BC5
:102D5000FF2099F0EE2009F4B5CF802F0F900F904F
:102D60000F900F900F90DF91CF911F910F91FF90D7
:102D7000EF90DF90CF900C944813EE2009F4B5CF7C
:102D8000802F0F900F900F900F900F90DF91CF91A9
:102D90001F910F91FF90EF90DF90CF900C94B313A1
:102DA000412F4F70602FC6010E940F1F0F900F9090
:102DB0000F900F900F90DF91CF911F910F91FF9087
:102DC000EF90DF90CF900C94D91A01112FC0FF2003
:102DD00069F10E94FF139FEFE0E7F2E09150E040BD
:102DE000F040E1F700C000000F900F900F900F909F
:102DF0000F90DF91CF911F910F91FF90EF90DF9097
:102E0000CF900C94B81E412F4F70602FC6010F90C9
:102E10000F900F900F900F90DF91CF911F910F9116
:102E2000FF90EF90DF90CF900C94121F0F900F90B7
:102E30000F900F900F90DF91CF911F910F91FF9006
:102E4000EF90DF90CF9008951F93CF93DF9300D042
:102E500000D01F92CDB7DEB7942F4983252F5A8318
:102E60006B837C838D834C815D81452B31F02F3FBB
:102E700031F481E09F3F19F403C081E001C080E09C
:102E8000182F117080FD31C049815A816B817C817E
:102E90008D810E948F1C292F22952F702C3030F4A9
:102EA0002A30A0F42250223030F022C02C30C9F059
:102EB0002F30B9F01DC0853A28F48430C0F4823038
:102EC00028F415C090E2980F983088F0883E30F4CE
:102ED000803E68F48450813A58F409C0803F41F440
:102EE00006C093FB112710F903C010E001C011E0E8
:102EF000812F0F900F900F900F900F90DF91CF9137
:102F00001F910895CF93DF9300D000D01F92CDB7CB
:102F1000DEB70F900F900F900F900F90DF91CF9131
:102F20000895CF93DF9300D000D000D0CDB7DEB7A7
:102F300026960FB6F894DEBF0FBECDBFDF91CF91BE
:102F400008951F93CF93DF93C091810216E0809183
:102F50008202C81799F0D0E01C9FF0011D9FF00D70
:102F60001124ED57FD4F408151816281738184812D
:102F700095810E9491172196C770E9CFDF91CF917B
:102F80001F9108954091B3025091B4026091B5022F
:102F90007091B6028091B7029091B8020C9491178B
:102FA000CF938091B80282958F7009F05FC08091B5
:102FB000B502882309F45AC080918102B09182023F
:102FC0007091B302A091B4024091B6025091B70241
:102FD00091E07F3F09F090E0692FC6E08B1709F47C
:102FE00045C04115510521F0AF3F21F020E003C05D
:102FF00021E001C0262F90E020FD35C0C89FF001E0
:10300000C99FF00D1124ED57FD4F21812A132BC0CC
:103010002081271328C02281211125C023813481DA
:103020002417350710F421503109241B350B283C97
:103030003105C8F42091B8022F7020612093B802A6
:1030400026E0289FF001299FF00D1124E857FD4F3D
:1030500080818F708061808383EB92E00E940314F3
:10306000CF910C94A11701968770B8CFCF91089596
:10307000AF92BF92CF92DF92EF92FF920F931F9386
:10308000CF93DF93CDB7DEB761970FB6F894DEBF6D
:103090000FBECDBF7C0185E0F701DE011D960190DA
:1030A0000D928A95E1F7D7014C9111965C91119799
:1030B0001296DC90129713960D911C9114973091F3
:1030C000B3026091B4028091B6029091B70200976A
:1030D00031F06F3F31F421E03F3F19F403C021E0AC
:1030E00001C020E0B22FB170BB2E20FD6EC1A090B8
:1030F000B502AA2009F4CCC02091B802081719071C
:1031000028F0F801E81BF90BCF0104C080959095D9
:10311000800F911FCC24C394883C910580F0C12C72
:10312000207F09F0A1C0702F198B088B6D2D898924
:103130000E94821783EB92E00E940314BDC0822F8D
:10314000807F09F056C0561315C0431313C0CD2C11
:10315000D11010C02F7020612093B8020E94C217B6
:1031600083EB92E00E9403148091B802D701159678
:103170008C935FC10115110531F05F3F31F481E09F
:103180004F3F19F403C081E001C080E080FD03C01F
:1031900081E08D2502C080E090E0B82FB170CB2E89
:1031A00080FF1CC0809181022091820236E082174C
:1031B00009F41CC190E0389FF001399FF00D1124F3
:1031C000ED57FD4F6181561306C06081461303C061
:1031D0006281D61203C001968770E9CFCD2CDD2025
:1031E00009F427C18091B80281608093B802C12C94
:1031F00020C1561308C0431306C0D11004C08091EB
:10320000B802D701B6C04D875E87DF86702F198B55
:10321000088B6D2D89890E942417882399F1DD2060
:1032200089F12091B802822F82958F7090E00297E9
:1032300074F08091B3029091B40298878F831986BD
:103240001B870A872C87CE0107960E94031486E00D
:10325000F701A3EBB2E001900D928A95E1F70E948D
:10326000D0170E94C21711C0561781F14D875E8793
:10327000DF86702F198B088B6D2D89890E9424178A
:10328000811138C0C7010E940314CC24C394D1C05B
:103290000817190708F446C0F801E81BF90BCF011D
:1032A000883C910508F443C0C12C702F198B088B02
:1032B0006D2D89890E948217E3EBF2E086E0DF0141
:1032C0001D928A95E9F70E94C217B3C04313CECF6F
:1032D000D110CCCF8091B802F7018583C7010E943D
:1032E000031486E0E3EBF2E0DF011D928A95E9F733
:1032F000CA2C9FC0DD2031F22091B802822F829526
:103300008F7090E002970CF4A2CF8091B30290915D
:10331000B4029A8389831B821D830C832E83CE0182
:10332000019693CF80959095800F911FB9CFCD2CAA
:10333000DD2009F4A7CF561333C0431331C02091C9
:10334000B80220FD24C0822F82958F70482F50E054
:1033500041155105E1F0D70115962C9315974F3083
:10336000510549F08F5F982F9295907F822F8F7033
:10337000892B15968C93C7010E94031486E0F701F0
:10338000A3EBB2E001900D928A95E1F79CCF86E025
:10339000F701A3EBB2E001900D928A95E1F749C0E5
:1033A0004D875E87DF86702F198B088B6D2D89897D
:1033B0000E94241781114BCF8091B80281608093C5
:1033C000B802C7010E94031434C0DD2009F45ACFAB
:1033D0004D875E87DF86702F198B088B6D2D89894D
:1033E0000E942417882309F44DCF31CF702F198BF9
:1033F000088B6D2D89890E948F1C292F22952F7093
:10340000223028F49F7039F0811105C00BC02430A0
:1034100028F49F7049F4805E883020F0C7010E9434
:103420000314BC2CCB2C05C0F7019581907F99F734
:10343000F9CF8C2D61960FB6F894DEBF0FBECDBFCD
:10344000DF91CF911F910F91FF90EF90DF90CF9080
:10345000BF90AF9008951F93CF93DF93CDB7DEB7A2
:103460002C970FB6F894DEBF0FBECDBF4F835887A1
:1034700069877A878B879C87CE0107960E943818C8
:103480008823D1F09F8188852A853B85232B31F0C5
:103490008F3F31F481E09F3F19F403C081E001C008
:1034A00080E080FD47C04F81588569857A858B858E
:1034B0009C850E9491173EC086E0FE013796DE0192
:1034C000119601900D928A95E1F7FF81E8856A8552
:1034D0007B856115710531F0EF3F31F481E0FF3FED
:1034E00019F403C081E001C080E080FD23C0209179
:1034F000820230E0C90101968770992740918102CC
:1035000050E084179507F1F1F983EA837D836C839A
:1035100096E0929FD001939FB00D1124AD57BD4FFF
:10352000FE01319601900D929A95E1F78093820207
:103530000E94A11716E08091810290918202891762
:1035400071F1189FC00111248D579D4F0E943818AA
:10355000882329F1E09181021E9FF0011124ED578B
:10356000FD4F4081518162817381848195810E94E8
:1035700091178091810290E001968770992780933E
:103580008102D9CF0E94FF13109282021092810211
:10359000E3EBF2E086E0DF011D928A95E9F72C96D5
:1035A0000FB6F894DEBF0FBECDBFDF91CF911F9154
:1035B0000895DF92EF92FF920F931F93CF93DF93C3
:1035C000FC01892B09F488C0E12CF12CDD24D39473
:1035D000EF0121968491853709F460C058F484374F
:1035E00008F04EC0843008F068C08130D1F08230DD
:1035F00071F172C0883709F45BC050F4863709F462
:1036000053C0873709F068C08E2D0E945E1D52C0DE
:103610009CE7980F903708F05FC08F770E94B31334
:103620004EC08F010E5F1F4FFE01849190E2980FF4
:10363000983050F48770FD2D01C0FF0F8A95EAF78E
:103640008F2F0E94641D15C00E94481314C08F0163
:103650000E5F1F4FFE01849190E2980F983068F43E
:103660008770FD2D01C0FF0F8A95EAF78F2F0E940A
:103670006A1D0E948B1DE80122C00E94B313FBCF7C
:10368000CF010296FE01C491CC2361F0EFE9FFE087
:103690003197F1F700C00000C150F6CFCF0102967C
:1036A000FE01F490EC010BC00E944E1DE82E07C0F5
:1036B0000E94611D0E948B1D02C00E9448138F2D25
:1036C000882341F0EFE9FFE03197F1F700C00000F7
:1036D0008150F6CFFE017CCFDF91CF911F910F91EA
:1036E000FF90EF90DF9008956093390370933A0351
:1036F00080933B0390933C030C94D91D08956093F1
:103700003D0370933E0380933F03909340030C94DA
:10371000D81D0F931F9300913D0310913E032091FC
:103720003F0330914003602B712B822B932B6093CE
:103730003D0370933E0380933F03909340031F919A
:103740000F910C94D81D0F931F9300913D0310917E
:103750003E0320913F033091400360237123822375
:10376000932360933D0370933E0380933F039093B4
:1037700040031F910F910C94D81D0F931F9300913C
:103780003D0310913E0320913F0330914003602799
:1037900071278227932760933D0370933E038093A4
:1037A0003F03909340031F910F910C94D81D60E04C
:1037B00070E0CB010C94741B0F931F9341E050E019
:1037C00060E070E08A019B0104C0000F111F221FFE
:1037D000331F8A95D2F7C901B8011F910F910C943C
:1037E000741B0F931F9341E050E060E070E004C051
:1037F000440F551F661F771F8A95D2F780913903B2
:1038000090913A03A0913B03B0913C038A019B0144
:10381000082B192B2A2B3B2BC901B8011F910F91A3
:103820000C94741B0F931F9341E050E060E070E034
:1038300004C0440F551F661F771F8A95D2F7409525
:103840005095609570958091390390913A03A091BD
:103850003B03B0913C038A019B01082319232A23CF
:103860003B23C901B8011F910F910C94741B0F9356
:103870001F9341E050E060E070E004C0440F551F2A
:10388000661F771F8A95D2F78091390390913A038A
:10389000A0913B03B0913C038A019B0108271927A3
:1038A0002A273B27C901B8011F910F910C94741B63
:1038B0000F931F930091390310913A0320913B031A
:1038C00030913C03602B712B822B932B1F910F9116
:1038D0000C94741B0F931F930091390310913A03BA
:1038E00020913B0330913C03602371238223932377
:1038F0001F910F910C94741B0F931F930091390328
:1039000010913A0320913B0330913C0360277127CB
:10391000822793271F910F910C94741B08958F9207
:103920009F92AF92BF92DF92EF92FF920F931F93FD
:10393000CF93DF9300D000D01F92CDB7DEB76B835B
:103940007C838D838A018C819D81892B31F01F3F7F
:1039500031F481E04F3F19F403C081E001C080E001
:1039600080FF03C080E090E04DC08B818823D1F1BF
:103970008090390390903A03A0903B03B0903C03B1
:1039800080913D0390913E03A0913F03B09140038D
:10399000882A992AAA2ABB2A8FE1E82EF12CD50180
:1039A000C4010E2C04C0B695A795979587950A94E7
:1039B000D2F780FD06C081E0E81AF10880F7D12C2B
:1039C00007C0DE2CB8018E2D0E94E71E019799F3E7
:1039D00088E0189FF0011124E754FD4FE00FF11D1E
:1039E000D08209C088E0189FF0011124E754FD4FF0
:1039F000E00FF11DD08009831A8369817A818D2DB2
:103A00000E94E71E0F900F900F900F900F90DF9184
:103A1000CF911F910F91FF90EF90DF90BF90AF90EB
:103A20009F908F9008952091110130911201F9011A
:103A300032969FEF40E05191851789F09F3F19F42E
:103A4000511101C0942F4F5F4630A9F79F3F39F0C5
:103A5000F901E90FF11D97FDFA9582830895089504
:103A6000E0911101F09112019F012A5F3F4F928175
:103A7000891301C012823196E217F307C1F7089546
:103A800081E090E0E0911101F0911201E80FF91F3F
:103A90001082019688309105A9F7089580914B0313
:103AA000089590914B03892B80934B030895809543
:103AB00090914B03892380934B03089580934B038C
:103AC000089510924B03089590914A03892B809397
:103AD0004A030895809590914A03892380934A036D
:103AE000089510924A030895809341030895109217
:103AF000410308958091110190911201FC013196CA
:103B00009C01285F3F4F80E0919191118F5FE217F8
:103B1000F307D1F70895E0911101F091120180911E
:103B20004B038083E0911101F0911201908180910B
:103B30004A03892B808380914103882361F0E091BF
:103B40001101F09112019081892B80830E947A1DCE
:103B500081111092410380911101909112010C94F6
:103B60005D1190933F0180933E0108958295982FB7
:103B7000937344E0949F900111248C7C86958695E4
:103B8000282B822F8575880F2A7A2695822B0895F7
:103B90000895CF93DF9300D000D01F92CDB7DEB74A
:103BA0000F900F900F900F900F90DF91CF9108958D
:103BB000089508950C94B41280E0089580916103F3
:103BC000843021F110924D0320E488E190E00FB69B
:103BD000F894A895809360000FBE2093600083B78F
:103BE000817F846083BF83B7816083BF7894889529
:103BF00083B78E7F83BF0FB6F894A895809160003D
:103C0000886180936000109260000FBE0895CF938A
:103C10000E9400130E9471070E940113C0E08C2FC4
:103C20000E942F08811104C0CF5FC031C1F701C0CD
:103C300081E0CF9108950E94B6120C94FF131F9259
:103C40000F920FB60F9211248F939F93AF93BF9350
:103C500080914D03811113C080914E0390914F03C9
:103C6000A0915003B09151034196A11DB11D8093C5
:103C70004E0390934F03A0935003B0935103BF9111
:103C8000AF919F918F910F900FBE0F901F9018953D
:103C900082E084BD93E095BD9AEF97BD80936E005E
:103CA00008952FB7F89480914E0390914F03A091FF
:103CB0005003B09151032FBF08952FB7F89460912E
:103CC0004E0370914F0380915003909151032FBF89
:103CD0000895CF92DF92EF92FF920F931F932FB729
:103CE000F89440914E0350914F03609150037091AE
:103CF00051032FBF6A017B01EE24FF248C0120E0D9
:103D000030E0C016D106E206F30610F44150510926
:103D10009A01281B390BC9011F910F91FF90EF9059
:103D2000DF90CF9008951F920F920FB60F9211243B
:103D30008F939F93AF93BF9380914E0390914F03C6
:103D4000A0915003B09151030196A11DB11D809324
:103D50004E0390934F03A0935003B0935103BF9130
:103D6000AF919F918F910F900FBE0F901F9018955C
:103D70000E94BA0FF89487E797E790930108809321
:103D8000000887E090EBDC0180936A0390936B035B
:103D9000A0936C03B0936D039CE088E10FB6F89498
:103DA000A895809360000FBE90936000FFCFE82F2E
:103DB000F0E088E0989FE00DF11D1124E052FF4FE4
:103DC0008491982F92959F708F7097700895CF93DC
:103DD000C82FCB010E94D71E40E1949F900111246F
:103DE000282B203831051CF080E090E016C0977039
:103DF000E92FF0E098E0C99FE00DF11D112494E057
:103E0000EE0FFF1F9A95E1F78F70E80FF11DEE0F8F
:103E1000FF1FE050F84985919491CF91089580E07B
:103E200090E0089508958091540380FF0BC0609145
:103E3000160185E0689FB001112475956795759509
:103E400067952BC081FF09C06091160185E0689FCE
:103E5000B00111247595679520C082FF07C060915D
:103E6000160185E0689FB001112417C09091550399
:103E70009923D1F060911501961788F720911601CA
:103E800085E0289F90011124929FA001939F500DDF
:103E9000112470E0CA010E94C5266038710540F403
:103EA0006115710519F406C065E070E0862F08956C
:103EB0008FE7089581E008958091540380FF08C042
:103EC0006091140170E0759567957595679521C0AF
:103ED00081FF06C06091140170E07595679519C067
:103EE00082FF04C06091140170E010C090915503EE
:103EF000992399F0609113019617A0F7809114010E
:103F0000899FC001112470E00E94C52660387105A8
:103F100040F46115710519F406C061E070E0862F68
:103F200008958FE7089581E00895803F21F40E946D
:103F3000131F819504C0813F29F40E94131F8093B1
:103F400058030895823F21F40E94131F819504C0F5
:103F5000833F29F40E94131F809357030895893FDC
:103F600019F40E945C1F05C08A3F31F40E945C1F57
:103F700081958093590308958B3F21F40E945C1F23
:103F8000819504C08C3F29F40E945C1F80935A03E2
:103F90000895843F21F480915603816017C0853FC6
:103FA00021F480915603826011C0863F21F48091F4
:103FB000560384600BC0873F21F4809156038860CC
:103FC00005C0883F31F48091560380618093560389
:103FD00008958D3F21F48091540381600BC08E3F82
:103FE00021F480915403826005C08F3F29F48091B1
:103FF00054038460809354030895803F39F4809182
:10400000580387FF6CC01092580369C0813F29F4A0
:10401000809158031816BCF362C090915703823FF9
:1040200029F497FF5CC01092570359C0833F19F4DD
:104030001916CCF354C0893F41F4809159031816E6
:104040000CF04DC0109259034AC08A3F29F4809168
:10405000590387FF44C0F6CF8B3F39F480915A0350
:1040600087FF3DC010925A033AC08C3F29F48091DB
:104070005A031816BCF333C0843F21F480915603D1
:104080008E7F17C0853F21F4809156038D7F11C02C
:10409000863F21F4809156038B7F0BC0873F21F42C
:1040A00080915603877F05C0883F31F48091560385
:1040B0008F7E8093560313C08D3F21F4809154036B
:1040C0008E7F0BC08E3F21F4809154038D7F05C0FD
:1040D0008F3F29F4809154038B7F80935403809108
:1040E000570381110EC08091580381110AC080913D
:1040F0005903811106C080915A03811102C01092A8
:104100005503089580914C0383FF7EC08DE395E0B5
:104110000E940A06809156031F928F9388E395E0D0
:104120009F938F930E94A30686E395E00E940A0660
:1041300080915703282F082E000C330B3F938F9349
:1041400083E395E09F938F930E94A30681E395E01C
:104150000E940A0680915803282F082E000C330B6A
:104160003F938F938EE295E09F938F930E94A306D7
:104170008CE295E00E940A0680915903282F082EB0
:10418000000C330B3F938F9389E295E09F938F93BD
:104190000E94A30687E295E00E940A0680915A03D6
:1041A000282F082E000C330B3F938F9384E295E069
:1041B0009F938F930E94A30681E295E00E940A06D6
:1041C000809155031F928F938EE195E09F938F937B
:1041D0000E94A3068CE195E00E940A068091540398
:1041E0001F928F9389E195E09F938F930E94A3067E
:1041F00086E195E00E940A068DB79EB74C960FB6F1
:10420000F8949EBF0FBE8DBF86E593E00E94A61175
:104210000E94511E909353038093520308951F935D
:10422000CF93DF9380915203909153030E94691EB4
:10423000AC0190915503992321F02091170130E0B2
:1042400006C0209118018AE0289F9001112442178E
:10425000530708F485C080915703C0915803D0914B
:10426000590310915A03811107C0C11175C0D111B2
:1042700073C0111171C074C09F3F19F09F5F90937C
:104280005503181624F40E94131F8093570380913E
:10429000570387FF05C00E94131F81958093570322
:1042A0001C1624F40E94131F809358038091580316
:1042B00087FF05C00E94131F81958093580360916A
:1042C0005703662331F1C0915803CC2311F1062E18
:1042D000000C770B880B990B0E94CC2523E333E36A
:1042E00043E35FE30E9430260E94942560935703C6
:1042F0006C2FCC0F770B880B990B0E94CC2523E3F6
:1043000033E343E35FE30E9430260E9494256093E9
:1043100058031D1624F40E945C1F8093590380915A
:10432000590387FF05C00E945C1F81958093590344
:10433000111624F40E945C1F80935A0380915A0343
:1043400087FF05C00E945C1F819580935A03DF910F
:10435000CF911F910C9482209F3F09F08FCFA0CF67
:10436000DF91CF911F910895E6E5F3E085E0DF014D
:104370001D928A95E9F710925503109254030895FF
:1043800080E697E00E940A061F9281E08F931F92B9
:1043900085E08F9382E197E09F938F930E94A3061D
:1043A0000F900F900F900F900F900F900895833003
:1043B000E9F128F4813061F0823009F10895853007
:1043C00009F462C008F449C0863009F474C0089545
:1043D00080911801262F30E0280F311D2F3F310525
:1043E00024F4680F6093180103C08FEF80931801C5
:1043F000809118011F928F938BE496E072C0809198
:104400001701262F30E0280F311D2F3F310524F4EE
:10441000680F6093170103C08FEF8093170180919D
:1044200017011F928F9389E396E05BC0809116017C
:10443000262F30E0280F311D2F3F310524F4680F5F
:104440006093160103C08FEF8093160180911601CF
:104450001F928F9386E296E044C080911501262F2B
:1044600030E0280F311D2F3F310524F4680F609391
:10447000150103C08FEF80931501809115011F92E4
:104480008F9381E196E02DC080911401262F30E0BA
:10449000280F311D2F3F310524F4680F609314015C
:1044A00003C08FEF80931401809114011F928F93AA
:1044B00088EF95E016C080911301262F30E0280F79
:1044C000311D2F3F310524F4680F6093130103C0A1
:1044D0008FEF80931301809113011F928F938DEDC5
:1044E00095E09F938F930E94A3060F900F900F90DB
:1044F0000F900895833081F128F4813059F0823093
:10450000D1F00895853009F449C0B8F1863009F436
:1045100056C0089580911801681720F4861B809377
:10452000180102C010921801809118011F928F93F8
:104530008EEC95E054C080911701681720F4861B1B
:104540008093170102C010921701809117011F92EA
:104550008F938CEB95E043C080911601681720F48F
:10456000861B8093160102C01092160180911601DD
:104570001F928F9389EA95E032C0809115016817E8
:1045800020F4861B8093150102C0109215018091C2
:1045900015011F928F9384E995E021C08091140149
:1045A000681720F4861B8093140102C01092140136
:1045B000809114011F928F938BE795E010C080913A
:1045C0001301681720F4861B8093130102C0109218
:1045D0001301809113011F928F9380E695E09F93C2
:1045E0008F930E94A3060F900F900F900F90089545
:1045F000CF93C82F1F928F9385E698E09F938F9358
:104600000E94A30681E090E0A0E0B0E0BC01CD01F3
:1046100004C0660F771F881F991FCA95D2F70E94A2
:104620007F1B0F900F900F900F90CF910C94FF1362
:10463000CF93873288F58E3108F00BC18E3009F4A4
:1046400087C0D8F4873009F460C08B3009F44FC0BC
:10465000863009F002C180914C03817F8E7F809368
:104660004C038AE698E00E940A0682E39BE00E94DF
:104670000A0681E080935C0346C0863109F4B0C02D
:1046800020F4803109F47AC0E8C0893109F491C07E
:104690008B3109F449C0E1C0883349F150F48932C3
:1046A00009F4D5C0853309F4D2C0873209F0D5C0EA
:1046B000CEC0833409F4CBC028F48A3308F4CDC0CB
:1046C0008953C8C0883409F0C8C00E94FF1381E232
:1046D0009BE00E940A062FEF83ED90E3215080407B
:1046E0009040E1F700C000000E94B81E0CC081E9B4
:1046F00098E041C088E09BE00E940A0680914C034C
:10470000816080934C03C1E0ADC080914C03C82F01
:10471000C17080FFEFCF84E19BE00E940A06809188
:104720004C03817F8E7F3FC090914C0391FBCC273F
:10473000C0F981E0C827892FC0FB81F980934C0321
:10474000CC2319F08BEF9AE029C08DEE9AE013C0CC
:1047500090914C0392FBCC27C0F981E0C827892FA8
:10476000C0FB82F980934C03CC2319F08EED9AE0C4
:1047700015C08EEC9AE00E940A06C5CF90914C03BA
:1047800093FBCC27C0F981E0C827892FC0FB83F9B0
:1047900080934C03CC2351F082EC9AE00E940A06ED
:1047A00080914C03816080934C035CC085EB9AE060
:1047B000E2CF86EA9AE00E940A0687E79AE00E9422
:1047C0000A0682E39AE00E940A068AE09AE00E94C2
:1047D0000A068AEB99E00E940A068FE899E0CBCF9F
:1047E00081E899E00E940A060E9451111F928F935E
:1047F00087E699E09F938F930E94A3068091100112
:104800001F928F9380E599E09F938F930E94A30658
:10481000809169021F928F938DE399E09F938F930C
:104820000E94A3060E945D1E9F938F937F936F93B8
:1048300086E299E09F938F930E94A3068DB79EB75F
:1048400042960FB6F8949EBF0FBE8DBF5CCF80E03E
:1048500001C08D510E94F82256CF84E299E00E9457
:104860000A06C0E08C2FCF91089580E00895CF9381
:10487000C82F80915C03813091F020F0823009F4E0
:1048800053C04AC1E0911101F0911201808184343A
:1048900089F0883879F0823209F040C10BC0E0918C
:1048A0001101F09112018081843421F0883811F0D7
:1048B000823261F48C2F0E945108811104C08C2F28
:1048C0000E9418232FC081E090E02CC08C2F0E9402
:1048D0003524811126C0C431E1F070F4CB3081F071
:1048E000C031D1F40E94C0218DE598E00E940A06F3
:1048F00082E080935C0315C0C93259F0C83361F47B
:104900008AE698E00E940A0681E698E00E940A067C
:1049100008C010925C0304C18BE598E00E940A066F
:10492000FFC081E08170FEC0C43228F5CE3108F0AE
:10493000C1C0CB30A1F1D0F4C73009F0D3C08EE1B3
:104940008093180182E3809317018AE08093160117
:1049500084E18093150188E08093140188E28093BC
:10496000130181E097E00E940A06BFC0C33149F1FC
:10497000C431C1F0B7C0CB3409F4A9C028F4C9329E
:1049800089F0C83361F0AEC0C13509F49EC0C235AC
:1049900009F499C0CE3409F0A5C06AE09EC00E9417
:1049A000C021A3C080915B03882319F010925B03A0
:1049B0009CC08EE097E00E940A0681E080935C0331
:1049C000B1C088EE96E00E940A0686ED96E00E944D
:1049D0000A06809118011F928F9383ED96E09F93B2
:1049E0008F930E94A30681ED96E00E940A068FEB4A
:1049F00096E00E940A06809117011F928F938CEB1C
:104A000096E09F938F930E94A3068AEB96E00E9404
:104A10000A068BEA96E00E940A06809116011F9210
:104A20008F9388EA96E09F938F930E94A30686EA6D
:104A300096E00E940A0685E996E00E940A068091A7
:104A400015011F928F9382E996E09F938F930E94A6
:104A5000A30680E996E00E940A068BE796E00E9492
:104A60000A06809114011F928F9388E796E09F9326
:104A70008F930E94A30686E796E00E940A068FE5C0
:104A800096E00E940A06809113011F928F938CE595
:104A900096E09F938F930E94A3068AE596E00E947A
:104AA0000A068DB79EB748960FB6F8949EBF0FBE04
:104AB0008DBF1BC0CE51EC2FF0E0EC5CFE4F80812F
:104AC00080935B0312C061E003C061E006C06AE04E
:104AD00080915B030E94D72108C080915B030E94F4
:104AE0007A2203C08FEF96E013C080915B03882386
:104AF00069F01F928F9389EF96E09F938F930E94A6
:104B0000A3060F900F900F900F9004C086EF96E0D1
:104B10000E940A0681E006C010925C0380E002C099
:104B200080E000CFCF9108950E949B256894B11139
:104B30000C942A2608950E940F2688F09F5798F01B
:104B4000B92F9927B751B0F0E1F0660F771F881F92
:104B5000991F1AF0BA95C9F714C0B13091F00E94AC
:104B60002926B1E008950C942926672F782F8827ED
:104B7000B85F39F0B93FCCF3869577956795B395D3
:104B8000D9F73EF490958095709561957F4F8F4F42
:104B90009F4F0895E89409C097FB3EF49095809547
:104BA000709561957F4F8F4F9F4F9923A9F0F92FF3
:104BB00096E9BB279395F695879577956795B79571
:104BC000F111F8CFFAF4BB0F11F460FF1BC06F5F57
:104BD0007F4F8F4F9F4F16C0882311F096E911C069
:104BE000772321F09EE8872F762F05C0662371F08A
:104BF00096E8862F70E060E02AF09A95660F771F9E
:104C0000881FDAF7880F9695879597F9089557FDCD
:104C10009058440F551F59F05F3F71F04795880F2A
:104C200097FB991F61F09F3F79F0879508951216C1
:104C300013061406551FF2CF4695F1DF08C016166D
:104C400017061806991FF1CF86957105610508941E
:104C50000895E894BB2766277727CB0197F9089535
:104C60000E9443260C94B4260E94A62638F00E9487
:104C7000AD2620F0952311F00C949D260C94A326CC
:104C800011240C942A260E94072670F3959FC1F3E5
:104C9000950F50E0551F629FF001729FBB27F00DEA
:104CA000B11D639FAA27F00DB11DAA1F649F66273F
:104CB000B00DA11D661F829F2227B00DA11D621F8E
:104CC000739FB00DA11D621F839FA00D611D221F48
:104CD000749F3327A00D611D231F849F600D211D2C
:104CE000822F762F6A2F11249F5750409AF0F1F0AF
:104CF00088234AF0EE0FFF1FBB1F661F771F881F18
:104D000091505040A9F79E3F510580F00C949D268C
:104D10000C942A265F3FE4F3983ED4F3869577956A
:104D20006795B795F795E7959F5FC1F7FE2B880FBD
:104D3000911D9695879597F9089597F99F6780E853
:104D400070E060E008959FEF80EC089500240A94DD
:104D50001616170618060906089500240A94121656
:104D60001306140605060895092E0394000C11F489
:104D7000882352F0BB0F40F4BF2B11F460FF04C036
:104D80006F5F7F4F8F4F9F4F089597FB072E16F44D
:104D9000009407D077FD09D00E94DF2607FC05D0DC
:104DA0003EF4909581959F4F0895709561957F4F42
:104DB0000895EE0FFF1F0590F491E02D0994AA1BB2
:104DC000BB1B51E107C0AA1FBB1FA617B70710F0F6
:104DD000A61BB70B881F991F5A95A9F78095909528
:0A4DE000BC01CD010895F894FFCF47
:104DEA000560010000FFE10871094E091809E4088D
:104DFA000142032808140A321E404D36227E04312D
:104E0A0004FB03D90365037E039703B0030000087C
:0E4E1A00000400020102030405060708090057
:106800008800EA44E944E244040005000600070069
:10681000080009000A000B000C000D000E000F001C
:1068200010001100120013001400150016001700CC
:10683000180019001A001B001C001D001E001F007C
:10684000200021002200230024002500260027002C
:10685000280029002A002B002C002D002E002F00DC
:1068600030003100000033003400350036003700BE
:10687000380039003A003B003C003D003E003F003C
:1068800040004100420043004400450046004700EC
:10689000480049004A004B004C004D004E004F009C
:1068A000500051005200530054005500560057004C
:1068B000580059005A005B005C005D005E005F00FC
:1068C0006000610062006300640065A100000000D8
:1068D000680069006A006B006C006D006E006F005C
:1068E0007000710072007300000087008A008B0046
:1068F000E000E100E200E3008140E500E600E7009F
:106900000100010001000100EA4401000100E2442D
:106910000100010001000100460001004A004B0097
:10692000010001004700480001000100E9440100A6
:106930000100010001000100010001003A003B00DC
:106940003C003D003E003F0040004100420043004B
:106950000100350001000100010044004500520023
:1069600001004900000050004F004C004D004E0057
:1069700051000100010001000100010001000100BF
:1069800001000100010001000100010001000100FF
:1069900001000100010001000100010001000100EF
:1069A00001000100010001000100010001000100DF
:1069B00001000100010001000100010001000100CF
:1069C00001000100010001000100010000000000C1
:1069D00001000100010001000100010001000100AF
:1069E00001000100010001000000010001000100A0
:1069F000010001000100010000E0010001000100B0
:00000001FF
